:10000000830100308A008B28FE0003088301ED0085
:100010000408EE000A08EF008A017008FF000B1DBB
:100020005E285630831203132018023E8400831783
:10003000000881070B11AD0B4C28AD0A3B2886192F
:100040004C28AD01AD0A4B28861D4928AE014C282D
:10005000A11935282F08463E840083132C08800000
:10006000AF0A2F08143A0319AF01AD01AD0AAC0174
:10007000AE01AA014C282E0803191F28013A0319C2
:1000800024282E080A3A0319282803108619031475
:10009000AC0C0430AD00AE0A2208031DA203FF30F1
:1000A000B007031CB10331083004031D80281F3042
:1000B000B0004B30B100A60AA016802883120313AB
:1000C0008C1E7B281A08EC0098186828181D6A28CE
:1000D0001812181621142017A01B80282908323E58
:1000E000840083136C088000A90A2908143A031DB0
:1000F0008028A90180288B1C80288B10A40AA014BA
:100100007F08F0006E0884006F088A006D08830085
:10011000FE0E7E0E0900223084006D30AB20A03030
:100120008400EF30AB20203084002230AB20203020
:10013000840056308317AB200730FD00FC30FC00F4
:10014000563084005A308317AF2083018A15842AE1
:1001500004068001840A0406031DA8280034F00068
:100160008A11BD208A118000840A040870060319D0
:100170000034B02883120313FC00FD1BC8287D1B2C
:10018000D0287D088A007C08FC0A0319FD0A820039
:1001900083137D1883177C08FC0A8400000808007C
:1002D6008312DF0083169B001C141A088312080081
:1002E6008312DE0083169C18752983125E08831616
:1002F6009B0083125D0883169A0003108B1B031460
:100306008B131C1555309D00AA309D009C141C11A2
:1003160003188B17831208008316031335088A15F2
:10032600EA21831636088A15EA212F308A15EA2132
:10033600831638088A15EA21831639088A15EA21B0
:1003460020308A15EA2183162B088A15EA2183169E
:100356002C088A15EA213A308A15EA2183162D08D7
:100366008A15EA2183162E088A15EA213A308A155B
:10037600EA2183162F088A15EA218A118316300886
:100386008A15EA2948308A15EA2174308A15EA2145
:10039600E10120308A15EA218A11E10A0D30610255
:1003A600031CCC29A708031DDA298430DB29C430B5
:1003B6008A150322BE308A11D52D8301E101E10A97
:1003C600BA308A11E72C8301E101B6308A11E72C95
:1003D6008301E301E40183162C088A1168242F3077
:1003E6008A15EA21E301E40183162B088A116824A1
:0A03F60020308A15EA21E301E4013A
:1004000083162F088A1168243A308A15EA21E301FD
:10041000E401831630088A1168243A308A15EA21EB
:10042000E301E401831631088A11682C8301DF009F
:10043000A92B8312A1100030A11801308316A5004A
:10044000831220118316251C272A8312201583125C
:100450005F08403A031DC32B702A83125F08403A9D
:100460008316031D742AA60A8312A114C32B8312B8
:100470005F08483A8316031D742AA60A83125F0890
:100480008316A400C32B83125F08623A8316031DF0
:10049000742AA60A83125F088316A406C32B83124C
:1004A0005F088316A4062508AB3E840083138312DD
:1004B0005F0880008316A50A25082F3A031DC32B69
:1004C000712A240883125F0683160319712AA60174
:1004D00083122015C32B83125F080D3A031D732A64
:1004E0008316A60AC32B8316A601C32BA60183126B
:1004F0005F080A3A031DC32B0430E000A708031D60
:10050000892A201E852A0630E000A01D892A0C3089
:10051000E00082308A1503226008F10026088A1163
:10052000B8278A117008DE0026080739DD008C2BF9
:100530008316CF08831203199F2A2016A02A20129F
:1005400083120313E301E40183164E088A11682421
:1005500020308A15EA21E301E40183164F088A114D
:10056000682420308A15EA218A11A011E22A5F301E
:100570008A15EA218A115F30C72A42308A15EA219A
:100580008A114730C72A41308A15EA2153308A152B
:10059000EA218A110C2B50308A15EA218A11483041
:1005A000DD2A50308A15EA218A114D30DD2A323099
:1005B000DA2A33308A15EA2144308A15EA218A1171
:1005C000A0150C2B83165008F0000530F100031025
:1005D000F00CF10BE72A70080739F200F301092B40
:1005E00072080319B72A013A0319B72A033A031903
:1005F000BD2A013A0319C32A073A0319CB2A013A43
:100600000319D12A033A0319D72A013A0319D92A1F
:100610000C2B73080319F02A20308A15EA218A115D
:10062000272B4F308A15EA218A114B30232B4F306C
:100630008A15EA218A114330232B5530202B4E3066
:100640008A15EA2156308A15EA218A113E2B0310B9
:100650008316510C0339F200F3013B2B7208031986
:10066000112B013A0319172B033A03191D2B013AD9
:1006700003191F2B3E2B730803192E2B20308A15CC
:10068000EA218A118316D11F472B4330482B48306B
:100690008A15EA218A11851E4F2B5230502B2030AB
:1006A0008A15EA218A11A7080319C32BC2308A15BB
:1006B00003228A11201AA019672B802B201A802B65
:1006C000A019832BA019862BA01DC32B892B5D0895
:1006D00003195E2B013A03195E2B033A0319602BB1
:1006E000013A0319602B073A0319622B013A0319E7
:1006F000622B033A0319642B013A0319642BC32BB1
:10070000EB218A11C32BE6218A11C32BE0218A1128
:10071000C32BC5218A11C32B5E08F000F43E0318D9
:10072000C32B0C3E031CC32B0030F00203308A00A5
:100730009D30700703188A0A8200982A982A982AFE
:10074000982A802B802B832B832B862B862B892B1F
:10075000892B8316031326080319192A013A031952
:100760002D2A033A0319372A013A0319432A073A73
:1007700003194F2A013A0319612A033A03196B2A14
:10078000013A0319762A831208008301E701630303
:10079000640465046604031DF12B0D2C83120313FE
:1007A0006308F0006408F1006508F2006608F300D1
:1007B00070080317A90271080318E32B710A0319C3
:1007C000F20A0319F30AAA0272080318EA2B720A42
:1007D0000319F30AAB027308031C730AAC02031378
:1007E000E70A03172C08803AF00003136608803AE2
:1007F0007002031D0A2C650803172B02031D0A2C27
:100800000313640803172A02031D0A2C0313630849
:1008100003172902031C112CCE2B031729080313DD
:10082000E70083160313230B162C1A2C8312E708F8
:100830000319232C83126708303E8A15EA218A1196
:100840008316A301A30A831208008301E90166034A
:100850006704031D392C492C831203136608831681
:10086000A902031CAA03831267088316AA02831233
:10087000E90A83162A08803AF00083126708803A52
:100880007002031D462C660883162902031C4D2C9A
:100890002C2C831629088312E90083120313E9081C
:1008A0000319552C8316A301A30A8312680B632C2A
:1008B0008316A3088312031D642CE908031D632C0F
:1008C00020308A15EA2983126908303E8A15EA2900
:1008D0008301E5008316A301831265088316A9002E
:1008E000AA018312640B7B2C6430E600E7016308E5
:1008F000E80025248A110A30E600E7016308E800D1
:1009000025248A11E601E60AE7016308E800252CA0
:1009100083160313A301A30A83126308F300640878
:10092000F4006508F500F0017A30F1004430F2007F
:100930008A1138278A1179278A1170088316A9002D
:100940007108AA0064308312E600E701E80125245B
:100950008A110A30E600E701E80125248A11E60140
:10096000E60AE701E801252C8301E3000317A9014A
:10097000AA01AB01AC010313E401E50103172B0845
:10098000AC002A08AB002908AA00A90103136308D8
:100990006407840083130008F000F101F201F30101
:1009A0000317A9047108AA047208AB047308AC0405
:1009B0000313E40A0319E50A6508803AF000803061
:1009C000700204300319640203180800BE2C83016E
:1009D000E200B4240317AC1F0F2D2908F0002A08E9
:1009E000F1002B08F2002C08F300F009F109F209DC
:1009F000F309F00A0319F10A0319F20A0319F30AB9
:100A00007008A9007108AA007208AB007308AC0056
:100A10000313610B0D2D5730152D5330152D031376
:100A2000610B142D4530152D4E308A15EA21031720
:100A30002908F0002A08F1002B08F2002C08F30026
:100A40008A119C27BA30F3005B30F4004A30F5007D
:100A50008A11F7267008A2007108A3007208A4008A
:100A60002208F0002308F1002408F2008A117927F7
:100A70008A117008A0007108A1000313E301E30AC2
:100A8000E401E40A031720086824DF308A15EA210C
:100A900003172108F1002008F0008A11AF27700821
:100AA000F3007108F4007208F50022308400831707
:100AB0008A11A326F3017030F4004230F50083124E
:100AC00003172230840083178A112F2783120317FC
:100AD0002208F0002308F1002408F2008A11792787
:100AE0008A117008A0007108A1000313E301E4015A
:100AF00003172008682427308A15EA2103172108E4
:100B0000F1002008F0008A11AF277008F300710887
:100B1000F4007208F5002230840083178A11A3269E
:100B2000F3017030F4004230F500831203172230D5
:100B3000840083178A112F27831203172208F000DD
:100B40002308F1002408F2008A1179278A1170081D
:100B5000A0007108A1000313E301E40103172008BA
:100B600068242E308A15EA2103172108F100200895
:100B7000F0008A11AF277008F3007108F4007208C2
:100B8000F5002230840083178A11A3268A1183126C
:100B9000031722080313E300031723080313E400D9
:100BA000031724080313E500882C8301E200B42412
:100BB0000317AC1FFC2D2D308A15EA218A1103176B
:100BC0002908F0002A08F1002B08F2002C08F30095
:100BD000F009F109F209F309F00A0319F10A0319FE
:100BE000F20A0319F30A7008A9007108AA00720832
:100BF000AB007308AC00002E2B308A15EA218A1155
:100C000083160313A30140308312E3004230E40053
:100C10000F30E5000030E601C5238A11A030E30063
:100C20008630E4000130E5000030E601C5238A117A
:100C30001030E3002730E4000030E501E601C52371
:100C40008A11E830E3000330E4000030E501E601FA
:100C5000C5238A118316A301A30A64308312E3001B
:100C6000E401E501E601C5232E308A15EA218A1147
:100C70000A30E300E401E501E601C5238A11E3013E
:100C8000E30AE401E501E601C5238A116D308A1506
:100C9000EA2984080319003472088000840371086B
:100CA00080008403700880000034F801710D720D1B
:100CB000F60076080319602EF80DF201F11708000E
:100CC000F001F101F2010034F810740D750DF70018
:100CD00077080319702E0318F814F501F4170800AB
:100CE000F701F301F401F501080076080319602EFD
:100CF000F113F80C760CF2000318F117492EF608E0
:100D0000031D932EF001F101F201492E7203031924
:100D1000F00A0319F10A0319F20A0310F20CF10C9C
:100D2000F00CF60A7F2EF208031D862E700871045F
:100D30000319822EF11B752EF6030319822E031060
:100D4000F00DF10D9A2E8030F5060008F000840AAF
:100D50000008F100840A0008F200C92E7608770224
:100D6000031CBD2E031908000310F20CF10CF00C4B
:100D7000F60A76087702B22E0310F50CF40CF30C89
:100D8000F70A7608770603190800BC2E8030F506AE
:100D9000840155266426AE26781CD62EF009F1096A
:100DA000F209F00A0319F10A0319F20AF81CE02EFD
:100DB000F309F409F509F30A0319F40A0319F50A0A
:100DC0007308F00774080318740FF1077508031807
:100DD000750FF207F801F21F7F2EF009F109F209F1
:100DE000F00A0319F10A0319F20A78147F2E84011C
:100DF00055266426F901FA01FB01F60803190800DB
:100E00007708031908007602773EF600780CF8069A
:100E10001830F5000310F90DFA0DFB0D7208031DD3
:100E2000192F74087102031D172F73087002031C19
:100E3000232F7308F0027408031C740FF102031CC3
:100E4000F20379140310F00DF10DF20DF50B0A2FDA
:100E50007908F0007A08F1007B08F2007F2E000884
:100E6000F000840A0008F100840A0008F200392F1B
:100E7000840155266426F901FA01FB010730F500CB
:100E80000310F40CF30C031C502F7008F9077108C1
:100E90000318710FFA0772080318720FFB0703108B
:100EA000F00DF10DF20DF50B402F0930F5005C2F20
:100EB0000310FB0CFA0CF90C0310F40CF30C031CDC
:100EC0006B2F7008F90771080318710FFA07720881
:100ED0000318720FFB07F50B582F7A307707F607C8
:100EE000780CF8067908F0007A08F1007B08F20027
:100EF0007F2E84015526F3018230F607F61B602E03
:100F0000F030F607F61B952F183076020318602E86
:100F1000F608031D8E2F7818EE270800F60303103D
:100F2000F00DF10DF20DF30D882F0310F20CF10C02
:100F3000F00CF60F952F8B2FF31FA12F7814EE27AF
:100F4000A22FF8018E30F6008401F30803197F2EDA
:100F50000310F30CF20CF10CF00CF60AA52FF201C1
:100F6000F11BF2037208F3009C2FF201F301A12F91
:100F7000F000F4010310FD307107031CDF2FF301B3
:100F8000F0307105031DC72F0430F300F10EF2019C
:100F90000310F30AF10D031CC92FF10C7108700244
:100FA0000318F000F20DF30BCD2FF41FD92FF20927
:100FB000F20A7208F41F0800F009F00A0800F10CA8
:100FC0000318E82FF10C031CF0010310F00C031CB4
:100FD00003107008F200F001F00DD52F0310FF3060
:100FE000F007F009031CF107F109031CF207F209ED
:100FF000031CF307F30908003234FF348034FF3454
:101060008301E400E40A6403AB3E840083130008B8
:10107000EA218A15E40A6403AB3E84008313000866
:10108000EA218A15DF30EA218A15E501640865073F
:10109000AB3E840083130008EA218A15E50A063076
:1010A0006502031C46282030EA218A152030EA21F7
:1010B0008A152030EA298301DD00042983125D08A6
:1010C0000D3A8316031D6728A201A20A0C292108E4
:1010D0001B3A0319A10121083B3E840083178312A8
:1010E0005D0880008316A10A0C29831221162115A0
:1010F000A1165D080A3A8316031D002921081B3A30
:10110000031DFF28831203173B08533A0319FF28D6
:10111000C23003228A159D284F308F285530EA218E
:101120008A154B30AF284830EA218A154C30AF2859
:101130004430EA218A155330AF2803173B08443A5C
:10114000031998280C3A03199328043A03198C2898
:10115000193A03198E283F30EA218A153F30EA21D7
:101160008A152030EA218A15C6284F30EA218A15CF
:101170004B30DB285630EA218A152D30DB285630DB
:10118000C2284330EA218A152B30DB2803173C089C
:101190002E3A0319B5286C3A0319BA280A3A0319EA
:1011A000C1281C3A0319BF28013A55300319B62843
:1011B000EA218A154E30EA218A152030EA218A1563
:1011C00003173D08EA218A1503173E08EA218A150C
:1011D00003173F08EA218A1503174008EA218A15F8
:1011E00003174108EA218A152030EA218A150317DE
:1011F0004208EA218A1503174308EA218A15831653
:101200000313A101A2010C29831603132208031959
:101210005E28013A03197528831208008301DD0056
:101220002B082F06031D1629031008002B08463E25
:10123000840083130008F0005D08840070088000BB
:10124000AB0A2B08143A0319AB01031408008301FD
:10125000DD0028082906031D2F290310080028088F
:10126000323E840083130008F0005D08840070089B
:101270008000A80A2808143A0319A80103140800DA
:10128000FB3083160313860083128514051505149D
:101290000608DB000510F030DB0505140608DA004F
:1012A00005105A0E0F39DB040B30831686008312AB
:1012B00085100230A2002208031D5B295B0808008C
:1012C00014308301A2002208031D6329FF30DE07CA
:1012D000031CDF035F085E04031908006029673000
:1012E000831603139900FA308312DE00DF016021B8
:1012F0009A019A019A010800CF30831603139900CE
:10130000FA308312DE00DF0160219A019A019A010E
:1013100008008301851005111E30DE00DF01602109
:101320000F30860530308604051405100530DE00C8
:10133000DF016021051405100230A2002208031D00
:101340009E29051405100530DE00DF0160210F30F5
:1013500086058616051405100230A2002208031D1A
:10136000AE29283003228A15083003228A150C3052
:1013700003228A150630032A83160313A00ACB29F9
:101380004030A000C7290E228A1583162008803E0F
:1013900003228A15D2292008103A0319C029403A9D
:1013A0000319C329831208008301EB000F3086055F
:1013B0006B08F0398604051405100F3086056B0E96
:1013C000F0398604051405100230A2002208031922
:1013D0000800E6298301EA000515D4298301DE000F
:1013E000F829DE0A5E038A116B218A15EA218A1523
:1013F00083120313DD035D0FF12908008301DA0076
:10140000EA218A15BC298301E4000511D4290130A1
:1014100003228A150330DE00DF0160298301DB012E
:10142000262A5B08C03E03228A154021DA005B08A9
:10143000C03E03228A152030EA218A155B08803ECF
:1014400003228A155A08EA218A15DB0A10305B024A
:10145000031C112AC03003228A1540308316A000D5
:1014600083120800073083019F0030308316850007
:101470000B3086008312A401A601A801A901A017C0
:10148000A11021102013AB01AF01A115A11221124F
:101490002111AD01AD0AAE01AC01AA0124308316C1
:1014A0009800903083129800673083169900831259
:1014B0009A019A019A01851120101F30B0004B301B
:1014C000B1002530A5008316A5016D2A25082D3E03
:1014D0008400831720308000A50A0E302502031CEB
:1014E000662AA501A1018112563083122018023EFE
:1014F00084008317000881008B1683168C160B1747
:101500000B168B1783120800322289218A15851E3B
:101510009F2AE830DE000330DF006021851E9F2A0D
:101520000630DD004E30EE214330DD001D308A11E3
:1015300073218A15D030DE000730DF0060211E30B5
:101540008A116B21A7001F308A116B218A15A30015
:1015500007228A151830DD000030EE21C03003224A
:101560008A150D30DD001030EE21D030DE0007305E
:10157000DF00602107228A15803003228A157C3023
:10158000EA218A15C03003228A157C30EA218A15A7
:10159000C23003228A15A3080430DD00031DD22ABD
:1015A0002030D32A2430EE21033023020318DB2A13
:1015B0002F30EA218A15023023020318E32A023071
:1015C000DD002830EE212308023A031DEB2A023009
:1015D000DD002A30EE21A708031DF52ACA300322B8
:1015E0008A150430DD002C30EE21823003221D30BC
:1015F0008A116B218A15433A031D0A2B0A30DD003C
:101600005830EE214C244830DD001D308A11732102
:101610008A151C2B0430DD005430EE21A308031979
:10162000132B7C218A150630DD005D30EE21D03091
:10163000DE000730DF00602107228A158515A01320
:10164000A1115C302721031C402BA308031D2D2B67
:101650005C088A1116228A152F2B5C08A625201DEE
:10166000402B823003228A150430DD007030EE21D9
:101670000430DD006330EE210630DD006830EE21FD
:10168000A708031D492B5C300E21031C492B5C0865
:101690005B20A01C542B260824060319542B240875
:1016A000A6005330DA005D2B20185A2B3D30DA00AB
:1016B0002D305D2B5E30DA005F30DB00A01C6B2B21
:1016C000A010803003228A15241C682B2A30692B35
:1016D0002B30EA218A15A01E212BA012C030032234
:1016E0008A15261C752B5A08762B5B08EA218A1569
:1016F0000A3026020318261C212B201BB12B823016
:1017000003228A150330DD007830EE210430DD003D
:101710007030EE210530DD007B30EE212030EA21F3
:101720008A152030EA218A1526081E3A0319211845
:10173000C22B07228A15823003228A150630DD006B
:101740004E30EE214330DD001D308A1173218A15A1
:10175000FA30DE00DF016021FA30DE00DF016021B7
:10176000842AA118C22B823003228A150430DD009E
:101770007030EE210530DD007B30EE210630DD00DB
:101780006830EE21A1102013A708031DF02B2119AA
:10179000DF2BC23003228A150330DD007830EE21C2
:1017A0000430DD007430EE210530DD007B30EE21A9
:1017B0002030EA218A152030EA218A15F02BA11A5F
:1017C000F02BC23003228A150430DD007430EE2184
:1017D0000530DD007B30EE210630DD006830EE2183
:1017E000A1122111212B8301DE00831203130C1E91
:1017F000F52B5E08990008004030F3234030F32BAE
:101800002430F3235030F3234D30F3234F30F323B0
:101810005430F3234730F3232C30F32B2430F323BD
:101820005030F3235230F3235730F3234930F3235E
:101830004930F3234C30F3234F30F3234730F32365
:101840002C30F32B0D30F3230A30F32B4730F323E6
:101850004730F3234130F3232C30F32B4730F3236D
:101860005330F3234130F3232C30F32B4730F32351
:101870005330F3235630F3232C30F32B4130F32332
:101880002C30F3235430F3232C30F3233130F32363
:101890002C30F3233030F32B7C218A1502302302C5
:1018A00003187A2C00248A154630F3234F30F32393
:1018B0005230F3232C30F3233030F32322248A15C3
:1018C000FA30DE00DF0160216F218A15FC238A15C2
:1018D0004330F3236630F3232530F32322248A1583
:1018E000DD01FA30DE00DF016021DD0A14305D0227
:1018F000031C712CA308031DBD2CFC238A15473043
:10190000F3236330F3230230F3232630F32322241E
:101910008A156430DE00DF016021FC238A15473020
:10192000F3236430F3230330F3232030F323222402
:101930008A156430DE00DF016021FC238A15473000
:10194000F3236530F323FF30F323DD30F323222428
:101950008A156430DE00DF016021FC238A154830DF
:10196000F3236230F3230130F3232B30F3232224BB
:101970008A156430DE00DF016021230BF52CFC2387
:101980008A154330F3236930F3230130F3232B30DE
:10199000F32322248A15FA30DE00DF0160217C2146
:1019A0008A1500248A1526248A153130F32322242F
:1019B0008A156430DE00DF01602100248A152E24A0
:1019C0008A153130F32322248A156430DE00DF01CA
:1019D000602100248A1536248A153130F32322240D
:1019E0008A156430DE00DF0160212308023A031DFE
:1019F00008000E248A1526248A153E248A152224DE
:101A00008A156430DE00DF0160210E248A152E2441
:101A10008A153E248A1522248A156430DE00DF01EF
:101A200060210E248A1536248A153E248A15222424
:101A30008A156430DE00DF0160298301E400E501DE
:101A40002A2DE50A6503AB3E8400831300082C3A77
:101A50000319E4036508AB3E840083138008031D6B
:101A6000E408031D212D6508080002301D25E20051
:101A7000AB3E840083130008EA218A152030EA2156
:101A80008A1501301D25E200302804301D25E300B1
:101A9000AB3E840083130008EA218A1503301D251C
:101AA000E300AB3E840083130008E200E30A303A0F
:101AB00003195C2D62085D2D2030EA218A15630828
:101AC00030284830EA218A157430EA218A15E3016A
:101AD0002030EA218A15E30A0D306302031C682DC9
:101AE000A708031D752D8430762DC43003228A1576
:101AF00008301D25E30009301D25F0007003E200C9
:101B00006308AB3E8400831300082D3A03198B2D24
:101B10002B30EA218A15620863020318982D6308A6
:101B2000AB3E840083130008EA218A15E30A8B2D5B
:101B30006D30EA298301E200393062020318A22DD8
:101B4000D030A32DC930E207620808008301E0000D
:101B5000DB2FA8018312A1108316281CB12D83123C
:101B6000A11400308312A11801308316A50083123E
:101B700020118316251CBE2D8312201583126008A8
:101B8000243A031DFE2F782E831260088316A400CA
:101B900083126008473A762E831260088316A406E3
:101BA00083126008503A8316031D7C2EA60A831206
:101BB000A114FE2FA601831260088316A4068312C7
:101BC0006008473A031DE72D04308316A6008312F0
:101BD00060085A3A031DFE2F07302F2EA6018312EC
:101BE00060088316A40683126008533A031DFB2D78
:101BF00005308316A60083126008473A031DFE2FA6
:101C000006302F2EA601831260088316A4068312C5
:101C10006008413A031D112E8316A801A80A0A3054
:101C2000A60083126008563A031DFE2F02303C2E98
:101C3000A601831260088316A40683126008413A45
:101C4000031DFE2F03303C2EA6018312600883166D
:101C5000A40683126008443A031DFE2F0830831641
:101C60003F2EA601831260088316A4068312600823
:101C7000413A031DFE2F04308316A8000A30A60047
:101C8000FE2F831260088316A406831260082C3A84
:101C9000762E2508AB3E84008313831260088000F3
:101CA0008316A50A831260082A3A0319782E600861
:101CB0008316A406FE2F831260089A25F000F00E0A
:101CC000F030F00570088316A700792E83126008A3
:101CD0009A258316A707270824060319792EA6013B
:101CE00083122015FE2F831260080D3A031D7B2EF0
:101CF0008316A60AFE2F8316A601FE2FA6018312C5
:101D000060080A3A031DFE2F0430E100A708031DF6
:101D1000912E201E8D2E0630E100A01D912E0C303C
:101D2000E100823003226108F10026088A11B827F9
:101D30008A157008DE0026080739DD00B52E851EDD
:101D4000A32E5230A42E20300317BA000313DF0154
:101D50005F082D3E840083170008EA218A15DF0AF8
:101D60000E305F020318CC2FA82E5E0803199F2E99
:101D7000013A03199F2E033A03199F2E013A0319C2
:101D80009F2ECC2F01301D25DF00A015D92E41300C
:101D90000317B3005330B4000313A011EB2E3230FD
:101DA0000317B3005330EA2E33300317B300443027
:101DB000EA2E5F08AB3E840083130008313A031912
:101DC000C72E033A0319CF2E013A0319D42E3F3000
:101DD0000317B300B400831603132B0883120317F1
:101DE000B900FE2F02301D25DF00AB3E84008313B7
:101DF00000080317AD0003135F0AAB3E8400000820
:101E00000317AE00FE2F05301D25DF002E2F4B30AF
:101E10000317B6004F30512F47300F2F44300317B0
:101E2000B6004630512F3130202F52300317B60004
:101E30005430512F46300317B6005230512F4530E1
:101E40000317B6005330512F4D300317B6004930F9
:101E5000512F53300317B6004D30512F5F08AB3E62
:101E6000840083130008303A0319072F013A03193D
:101E70000C2F033A03190E2F013A0319132F073AB7
:101E80000319152F013A03191A2F033A03191F2FAB
:101E9000013A0319242F0F3A0319292F3F30031752
:101EA000B600B70006301D258313DF00AB3E84006B
:101EB00000080317B00003135F0AAB3E840000085C
:101EC0000317B1003008303A031D6A2F3108303A49
:101ED00003196D2F031320166F2F03132012831283
:101EE0000313A708031D882F5E08063A03198E2FD7
:101EF000013A03198E2F0F3A0319932F013A031950
:101F0000932F033A0319982F013A031D0800982FC5
:101F1000C23003228A159B2FA01D912F35258A15CB
:101F2000FE2FA01D962F45258A15FE2FA01DFE2FE2
:101F300061258A15FE2F5D08023A03198C2F013A9C
:101F400003198C2F073A0319912F013A0319912F86
:101F5000033A0319962F013A0319962FFE2F831285
:101F6000A708031DBB2F5E08043A0319C12F013ACD
:101F70000319C12FFE2FC23003228A15C52F201E40
:101F8000FE2F8A118F218A15FE2F5D080319BF2F9E
:101F9000013A0319BF2FFE2F83162808013A0319AF
:101FA000C22E033A0319F22E013A0319032F073AFE
:101FB0000319AF2FFE2F831603132608F000F03EFF
:101FC0000318FE2F103E031CFE2F0030F0020F30CE
:101FD0008A00EE30700703188A0A8200A92DC42DEA
:101FE000CC2DDA2DEE2D022E182E242E312EFE2F82
:101FF000412E492E5B2E662E732E7E2E8301080005
:02400E00423F2F
:10420000470050005300200031002E0033002000F2
:1042100042002E00560045004C004C004500200096
:104220002800430029003200300030003800200010
:104230005000360034003800410043000000000008
:104240002000420049004E004E004D004500410054
:104250004D005400520043005400430058004F00EA
:10426000200020002000200020002000200020004E
:10427000200020002000200020002000200020003E
:10428000200020002000200020002000200020002E
:1042900020002000200020002000200052004500C7
:1042A000530045005400200048004F0054002000F7
:1042B00043004F004C0044002000530054004100D4
:1042C0005200540020004300520043002000200010
:1042D0004500720072006F00720020002000200074
:1042E0004700500053002000430058004F002000BA
:1042F0004E006F0020004C0069006E006B00200033
:00000001FF
